:1000000012C02AC029C028C027C026C02CC024C0C6
:1000100023C022C021C020C01FC01EC01DC01CC0E4
:100020001BC01AC019C011241FBECFEDCDBF10E0F8
:10003000A0E6B0E0ECE4F1E002C005900D92A0363D
:10004000B107D9F710E0A0E6B0E001C01D92A936D3
:10005000B107E1F704D078C0D3CF0895089557D001
:10006000FCDFFCDFFECF1F920F920FB60F92112420
:100070002F933F934F935F936F937F938F939F93B0
:10008000AF93BF932091640030916500409166006A
:100090005091670070916800DA01C9010296A11DB4
:1000A000B11D672F6A5F6D3730F06D57DA01C901F6
:1000B0000396A11DB11D6093680080936400909326
:1000C0006500A0936600B0936700809160009091F6
:1000D0006100A0916200B09163000196A11DB11D65
:1000E0008093600090936100A0936200B0936300DE
:1000F000BF91AF919F918F917F916F915F914F9140
:100100003F912F910F900FBE0F901F9018957894EC
:1001100080B7836080BF83B7877F83BF83B7887FC3
:10012000836083BF89B7826089BF8EB5887F8EBDAB
:100130008FB58C7F81608FBD8EB5877E8EBD8EB56D
:0C014000887F83608EBD0895F894FFCF87
:00000001FF
